:020000040000FA
:04000000B6EF00F067
:0400080004EF00F011
:080018000CEF00F09CEC00F07D
:100020008490030E46EC00F099EC00F084828492F8
:1000300090EC00F08482849290EC00F08490020EA8
:1000400046EC00F090EC00F0280E4CEC00F0100EA6
:100050004CEC00F0060E4CEC00F00C0E4CEC00F0FA
:10006000010E4CEC00F099EC00F01200800E4CEC0C
:1000700000F01200C00E4CEC00F01200940E4CEC9C
:1000800000F01200D40E4CEC00F01200806E84825E
:10009000849290EC00F01200096E0938849046ECCE
:1000A00000F00950849046EC00F01200300F096E09
:1000B0000938848046EC00F00950848046EC00F05A
:1000C00012000C6E70EC00F00A5056EC00F00B3889
:1000D0000F0B56EC00F00B500F0B56EC00F012001B
:1000E0000A6A0C380C240F0BD8B2160FD8B2060FC0
:1000F000060FD8A2FA0F0CB81B0FD8A2FA0F0CBA31
:10010000300F0CBC600F0CBE200F600F0A360AA027
:10011000A00F0B6E0CBE0A2A1200530E91EF00F0D6
:10012000350E006E002E92EF00F01200FA0E9DEFD9
:1001300000F0050E9DEF00F0280E016EA4EC00F01B
:10014000012E9EEF00F012008DEC00F08DEC00F01F
:100150008DEC00F08DEC00F0120096EC00F096ECC7
:1001600000F096EC00F096EC00F01200C168F26A24
:10017000926A936A946A956A966A0EEC00F0839C80
:10018000838CADEC00F0839C96EC00F0838A838E28
:100190008398EFEC03F0E2EC03F0E2EC03F00D687F
:1001A0000E680E50E3EC03F0D8900E3602E3CF0E4B
:1001B0000E1A0D2ED1EF00F036EC00F0000E61ECBF
:1001C00000F0ADEC00F0870E106EFDDA076A086AE9
:1001D000100E0E6EFDDA116E1130073608360E2E37
:1001E000F9D76D0E0862C2D7500E0762BFD7980EBE
:1001F0001062EAD736EC00F0010E61EC00F0ADECD5
:1002000000F0F00EE3EC03F08388EFEC03F083845E
:10021000010EE3EC03F0832AE2EC03F0F2EC03F0CE
:10022000E2EC03F0832A580EE3EC03F08306E2ECE1
:1002300003F0832A280EE3EC03F08306050EE3ECBB
:1002400003F0832A800EE3EC03F08306020EE3EC56
:1002500003F0832A080EE3EC03F0EFEC03F03C0E0E
:10026000E3EC03F0832A500EE3EC03F0832A9B0EA9
:10027000E3EC03F0832A180EE3EC03F0832AF40E78
:10028000E3EC03F0832A520EE3EC03F0F2EC03F00C
:10029000040EE3EC03F0832A080EE3EC03F08390F2
:1002A000839483868382C00EE3EC03F0832AE2EC1E
:1002B00003F0F2EC03F0E2EC03F0832A200EE3EC0F
:1002C00003F08306E2EC03F0832A480EE3EC03F02C
:1002D0008306010EE3EC03F0832A080EE3EC03F03F
:1002E000838083948386838273DA380B0009D8B4C1
:1002F00001D094D7EFEC03F083866ADA076E832A85
:1003000067DA086E08BEECD708BCDAEF03F0070E18
:10031000081610EE0DF008C0DAFF07C0D9FFEFECA9
:1003200003F056DAE66EDD52D966F9D7DA66F7D70A
:1003300010EE19F030EC00F036EC00F0E75061EC14
:1003400000F0080EE66236D2E75061EC00F0000ED5
:10035000E76404D0060EE7622DD2C6D13EEC00F071
:1003600010EE27F0E65061EC00F02E0E57EC00F096
:10037000E65061EC00F02E0E57EC00F0E65061EC18
:1003800000F02E0E57EC00F0E65061EC00F03AEC75
:1003900000F0E65061EC00F02E0E57EC00F0E65055
:1003A00061EC00F02E0E57EC00F0E65061EC00F02E
:1003B0002E0E57EC00F0E65061EC00F010EE24F049
:1003C000010EE76201D07FD1060EE762F3D1000E85
:1003D0003162F0D1500E3262EDD13CA015D000EE6A
:1003E00000F010EE31F030EC04F010EE2FF000EEE3
:1003F00031F030EC04F010EE00F000EE2FF030ECB5
:1004000004F03C883C9015D03CA233D000EE00F0C4
:1004100010EE31F030EC04F010EE2FF000EE31F081
:1004200030EC04F010EE00F000EE2FF030EC04F0B1
:100430003C8810EE33F000EE37F02CEC04F03A2A52
:10044000000E39223822372233363432353A3336E9
:100450001F6A206A35EC04F00F0E3B16500E3B125B
:10046000086A1D6A360E076E280E1E6E54EC04F0E4
:100470009FD13CA89FD13C883C803C923C943C96C8
:100480003C9A000E1D6204D0280E1E6201D092D14B
:100490003B380F0B040D20EE2FF0F350D926F4500B
:1004A000DA22000EF66E0A0EF76E000EF86E0900E4
:1004B000F5500009D8B403D0DE627CD1F8D7200E05
:1004C000DF620DD0260EF66E090EF76E000EF86E86
:1004D0000900F5500009D8B4DBD7DE6EF9D7DACFC2
:1004E00005F0D9CF06F000EE00F010EE31F030EC60
:1004F00004F010EE2FF000EE31F030EC04F010EECE
:1005000000F000EE2FF030EC04F010EE33F000EECF
:1005100000F02CEC04F000EE33F010EE37F02CEC91
:1005200004F010EE00F000EE37F02CEC04F01DC0EB
:1005300000F01EC001F0280E015E000E005A0150AE
:100540003A2600503922000E3822372230EC00F0D3
:1005500036EC00F010EE00F0E65061EC00F0E650F2
:1005600061EC00F010EE43F00F0E3B16500E3B1204
:10057000060EF66E0A0EF76E000EF86E05C0DAFF74
:1005800006C0D9FF0900F5CF00F000660DD0640E5B
:10059000006E090E016E000E026E320EF66E090E2E
:1005A000F76E000EF86E2CD00900F550DE6207D011
:1005B000002EFAD7200EDE6201D016D0002A0004E9
:1005C000F626000EF722F6CF00F0F7CF01F0090073
:1005D000F55000260900F550012200C0F6FF01C0C9
:1005E000F7FF09000900CAD7F6CF00F0F7CF01F0F6
:1005F000F8CF02F0C00EF66E090EF76E000EF86E20
:100600000900F5500009D8B402D0E66EF9D700C051
:10061000F6FF01C0F7FF02C0F8FF0900F5CF00F0B8
:100620000900F5CF01F00800F5CF04F00900740EC1
:10063000046224D03C0EF56221D009003F0EF56221
:1006400001D004D00A003C0EF56E18D00900070E48
:10065000F5140FEE80F0E926E90609000F0EF514F7
:10066000036E032AEFCFF5FFF532032EFDD7F56AAF
:10067000300EF522030E005E000E015AF5CFE6FFA4
:100680000006000E015A0066D1D70166CFD7E76A8F
:1006900020EE43F0D950E15EDA50E25A280EE1260E
:1006A000000EE222E2CF1DF0E1CF1EF00E0EE12699
:1006B000000EE222E2CF08F0E1CF07F035EC04F0C3
:1006C00054EC04F075D010EE2FF0080EE76272D0F3
:1006D00010EE2FF0E66A35EC04F0080E3126D8B0A3
:1006E000322AD8B4312A64D03EEC00F010EE29F062
:1006F000E65061EC00F02E0E57EC00F0E65061EC95
:1007000000F02E0E57EC00F0E65061EC00F02E0EDB
:1007100057EC00F0E65061EC00F03AEC00F010EE1F
:1007200033F0E65061EC00F02E0E57EC00F0E6508E
:1007300061EC00F02E0E57EC00F0E65061EC00F09A
:100740002E0E57EC00F0E65061EC00F010EE21F0B8
:10075000000EE6622FD0010EE6622CD010EE33F0D0
:10076000C00EE66227D0A80EE66224D0010EE66233
:1007700021D0630EE6621ED010EE21F0E66A020E72
:10078000E66E00EE2DF028EC04F02CEC04F000EE08
:1007900023F012EC04F01FEC04F000EE0DF010EE6C
:1007A00013F028EC04F012EC04F02A0E076E086A2D
:1007B000F6EC03F0F2EC03F005D8832A400E03D8E0
:1007C00070EF01F0000E816E839EAADC838E120012
:1007D0009368839AA5DC8150838A936A1200F00E95
:1007E000831612000F0E831283901200EFEC03F0B9
:1007F0000750E9DF0850E7DFE5DFE4DF10EE0DF03A
:1008000008C0DAFF07C0D9FFE650DDDFDD52D96648
:10081000FBD7DA66F9D7030E071401E11200D2DF25
:10082000072AF9D73C0EEE6E500EEE6E9B0EEE6E62
:10083000180EEE6EF40EEE6E520EEE6E1200C00E3C
:10084000EE6EA80EEE6E010EEE6E630EEE6E1200F0
:10085000E6CFEEFFE6CFEEFFE6CFEEFFE6CFEEFF10
:10086000E6CFEEFFE6CFEEFF120000EE0DF010EE49
:1008700013F0EEDFD7DF00EE2BF010EE27F0ECDF09
:1008800000EE27F0DCDF1200D890DA32D932D890AF
:10089000E6500222E6500322DD50D966F9D7DA6627
:1008A000F7D7000E02221200026A036A10EE27F048
:1008B000DA6A080ED96E44EC04F024500322000ECC
:1008C00002221DC000F01EC001F0140E015E000ED9
:1008D000005A10EE00F0DA6A020ED96E44EC04F011
:1008E00010EE2FF000C0DAFF01C0D9FFD92A3F6A0D
:1008F000406A44EC04F0031E021E02C03FF003C035
:1009000040F0026A036ADA6A140ED96E256A266A12
:1009100010EE1BF044EC04F0031E021E02C025F092
:1009200003C026F01200696E6465782E68746D6CE1
:100930002000485454502F312E3020343034204E73
:100940006F7420466F756E640A436F6E74656E74C3
:100950002D547970653A20746578742F68746D6CC5
:100960000A0A000059003C48544D4C3E3C48454161
:10097000443E3C5449544C453E343034204E6F7410
:1009800020466F756E643C2F5449544C453E3C2FB5
:10099000484541443E3C424F44593E3C48313E3438
:1009A0003034204E6F7420466F756E643C2F483192
:1009B0003E3C2F424F44593E3C2F48544D4C3E0044
:1009C000485454502F312E3020323030204F4B0AB3
:1009D0005365727665723A20504943313846343552
:1009E00032202B2033434F4D203343353039620AB8
:1009F000436F6E74656E742D547970653A200000F3
:100A0000474554202F00096D656E752E68746D6C16
:100A10005904746578742F68746D6C0A0A3C21441B
:100A20004F43545950452048544D4C205055424C4A
:100A3000494320222D2F2F5733432F2F4454442036
:100A400048544D4C20342E3031205472616E7369FD
:100A500074696F6E616C2F2F454E223E0A3C68749C
:100A60006D6C3E3C686561643E0A3C6D6574612056
:100A7000687474702D65717569763D22436F6E746C
:100A8000656E742D547970652220636F6E74656E87
:100A9000743D22746578742F68746D6C3B63686173
:100AA000727365743D69736F2D383835392D312275
:100AB0003E0A3C7469746C653E5049433138663473
:100AC0003532202B2033434F4D20334335303942CC
:100AD000202D20576562736572766572202D3C2F3C
:100AE0007469746C653E0A3C6D657461206E616D5D
:100AF000653D224B6579776F7264732220636F6E58
:100B000074656E743D225049433138663435322C59
:100B1000203343353039422C207765627365727615
:100B20006572223E0A20203C7374796C65207479CA
:100B300070653D22746578742F637373223E0A09D1
:100B4000613A686F7665727B636F6C6F723A72653B
:100B5000643B20746578742D6465636F7261746999
:100B60006F6E3A6E6F6E653B207D0A20203C2F73BE
:100B700074796C653E0A3C2F686561643E0A0A3CE4
:100B8000626F6479207374796C653D226D61726760
:100B9000696E3A3070783B2220746578743D222368
:100BA00030303030303022206267636F6C6F723DBE
:100BB000222345304530453022206C696E6B3D2242
:100BC000233030303046462220766C696E6B3D22F1
:100BD000233830303038302220616C696E6B3D2212
:100BE00023464630303030223E0A0A3C7461626C43
:100BF00065207374796C653D22626F726465723A28
:100C000020736F6C69642032707820677265656E3E
:100C10003B2220626F726465723D22302220636540
:100C20006C6C73706163696E673D2230222063656E
:100C30006C6C70616464696E673D22352220626766
:100C4000636F6C6F723D2223424244444646222029
:100C500077696474683D2231303025222073756DC8
:100C60006D6172793D22223E0A3C74723E0A3C74E8
:100C700064206E6F7772617020616C69676E3D727F
:100C8000696768743E0A4D656E750A3C2F74643E50
:100C90000A3C7464207374796C653D22636F6C6FD9
:100CA000723A20677265656E22206E6F777261708E
:100CB0003E0A7C0A3C2F74643E3C7464206E6F775D
:100CC0007261703E0A3C6120687265663D222E2F7B
:100CD00064656D6F2E68746D6C2220746172676537
:100CE000743D2264796E616D6963223E44656D6F67
:100CF0003C2F613E0A3C2F74643E0A3C74642073AE
:100D000074796C653D22636F6C6F723A206772650F
:100D1000656E22206E6F77726170203E0A7C0A3CFD
:100D20002F74643E3C7464206E6F777261703E0A6B
:100D30003C6120687265663D222E2F6764656D6F89
:100D40002E68746D6C22207461726765743D226434
:100D5000796E616D6963223E44656D6F322028773C
:100D6000697468207069637475726573293C2F61BA
:100D70003E0A3C2F74643E0A3C7464207374796CA0
:100D8000653D22636F6C6F723A20677265656E22F3
:100D9000206E6F77726170203E0A7C0A3C2F74646B
:100DA0003E3C7464206E6F777261703E0A3C612035
:100DB000687265663D222E2F696E666F2E68746DAF
:100DC0006C22207461726765743D2264796E616D76
:100DD0006963223E4D6F726520696E666F3C2F61BC
:100DE0003E0A3C2F74643E0A3C2F74723E0A3C2F2C
:100DF0007461626C653E0A3C7461626C6520616C72
:100E000069676E3D2263656E74657222206865694C
:100E10006768743D22383025223E0A3C74723E3C9D
:100E200074643E3C68313E50494331386634353253
:100E3000202B2033434F4D20334335303942202D72
:100E40002057656220536572766572202D3C2F68AD
:100E5000313E3C2F74643E3C2F74723E3C2F626FD7
:100E600064793E3C2F68746D6C3E0A05302E6769CC
:100E7000668F01696D6167652F6769660A0A474970
:100E80004638396112001200D53000F5F5F5E8E872
:100E9000E8F9F9F9D2D2D2F66088C9C9C97676766E
:100EA0006262629E9E9EF35F87D6D6D65B5B5BCA0C
:100EB000CACAFB678FF9638BEA5E83EE5D84CB540D
:100EC00074FA6A8FB67587DE7591FA678D848484AB
:100ED000FA658CFA96B1F96C92F96C91F8628AE82D
:100EE0005C81854556F984A3B94F6BE6A6B7D45DFE
:100EF0007D4C4C4CD56D88F06086F56188F4648A31
:100F0000F17A9AF35F86414141FBC0D0FBC7D5FB24
:100F1000678EF76289CCCCCCF56087FFFFFF0000BD
:100F200000000000000000000000000000000000C1
:100F300000000000000000000000000000000000B1
:100F4000000000000000000000000021F904010082
:100F50000030002C00000000120012000006A1402A
:100F60009870482C1A612B4FA651D19C4001C11199
:100F700023B96C5AD89689320014312C478BF02A49
:100F8000BF08A511C32B54491C64B39C3419486194
:100F90009E4B4BCE7F85100142191B717D650F065C
:100FA0000A420D7B866609072E42158D8E2F090B8E
:100FB00005421A958E1C9942279D86119142202642
:100FC000857D101D89420114258E281F2280420232
:100FD000032324AB1F29167643000C13210F0909A4
:100FE0001C111D22166B4500030806070B0B070694
:100FF000085D4702010A2E05052E0A5147E64741C2
:10100000003B05312E6769669401696D6167652F44
:101010006769660A0A47494638396112001200D5E5
:101020003300E8E8E8F5F5F554F27D53EF7C5B5BBF
:101030005BC9C9C9626262F9F9F9D2D2D2D6D6D6F1
:1010400061F688FAFAFA60F5875DF68556F47F5006
:10105000E4774AC76A5BF784B4F9C6CACACA51EAD8
:101060007954F17E85858564D3813F7F50A0A0A00F
:101070005AF68358F6817676769E9E9E77777770BD
:10108000EE9189F8A654EC7B4C4C4C6DDC8957F002
:101090007F57F58153D175A0E4B246B36271B48233
:1010A00052E67977F699D3D3D35AF784424242CBAA
:1010B000CBCB55F37FCCCCCC53F17DFFFFFF0000B1
:1010C0000000000000000000000000000000000020
:1010D0000000000000000000000000000000000010
:1010E000000021F90401000033002C000000001270
:1010F0000012000006A6C09970482C1A679295222B
:10110000A2617C4E80C311D4D83860581869840815
:101110001441AD124C202BCB0495CBC42B94344AF4
:1011200064B33C94424867AB0D4CCE97993A004269
:101130000A0E717D652A1C0942117B866603063101
:10114000421A8D8E32030405420C958E0F99421F70
:101150009D861091422724857D14181E8A33002312
:10116000158E03282219813307081721AB282E1664
:101170002C0B43011329262A03030F101822162FC4
:101180006CC5081D1C060404061E192CD344070058
:1011900009310505310900C447EB4641003B0A69A6
:1011A0006E6465782E68746D6C7F01746578742F39
:1011B00068746D6C0A0A3C21444F435459504520D1
:1011C00048544D4C205055424C494320222D2F2F3E
:1011D0005733432F2F4454442048544D4C20342E31
:1011E0003031204672616D657365742F2F454E2234
:1011F0003E0A3C68746D6C3E0A3C686561643E0A58
:101200003C7469746C653E504943313866343532FC
:10121000202B2033434F4D20334335303942202D8E
:101220002057656220736572766572202D3C2F749D
:1012300069746C653E0A3C2F686561643E0A3C66D1
:1012400072616D6573657420726F77733D22313002
:10125000302C2A2220626F726465723D2230222077
:101260006672616D65626F726465723D2230223E06
:101270000A3C6672616D65206E616D653D2266692E
:1012800078656422206672616D65626F7264657252
:101290003D223022207363726F6C6C696E673D2251
:1012A0006E6F22207372633D226D656E752E6874B9
:1012B0006D6C222069643D22666978656422206E27
:1012C0006F726573697A653E0A3C6672616D65206E
:1012D0006E616D653D2264796E616D696322206681
:1012E00072616D65626F726465723D223022207397
:1012F00072633D2264656D6F2E68746D6C22206987
:10130000643D2264796E616D696322206E6F72653F
:1013100073697A653E0A3C2F6672616D6573657408
:101320003E0A3C2F68746D6C3E0A0964656D6F2E31
:1013300068746D6CB402746578742F68746D6C0A8F
:101340000A3C68746D6C3E3C686561643E3C6D654A
:10135000746120687474702D65717569763D2243DF
:101360006F6E74656E742D547970652220636F6E94
:1013700074656E743D22746578742F68746D6C3B6F
:10138000636861727365743D69736F2D38383539E0
:101390002D31223E3C6D65746120687474702D653A
:1013A000717569763D2252656672657368222063A5
:1013B0006F6E74656E743D2234223E3C2F68656109
:1013C000643E0A3C626F647920746578743D233012
:1013D0003030303030206267636F6C6F723D234570
:1013E0003045304530206C696E6B3D2330303030F5
:1013F000464620766C696E6B3D233830303038308D
:1014000020616C696E6B3D234646303030303E0AB9
:101410003C68723E3C703E54686973207765627325
:101420006974652069732062726F756768742074CF
:101430006F20796F7520627920612077656273650E
:101440007276657220746861742069732072756E9B
:101450006E696E67206F6E206120504943313846B7
:1014600034353220636F6E6E656374656420746F0B
:1014700020612033434F4D203343353039422065BE
:10148000746865726E657420636172642E3C2F709F
:101490003E0A3C703E42656C6F7720796F75206321
:1014A000616E2073656520776869636820696E7076
:1014B0007574206F66207468697320504943313811
:1014C00066343532206973206869676820283129BD
:1014D000206F72206C6F77202830292E3C2F703EB1
:1014E0003C68723E0A3C5052453E0A504F525441AD
:1014F000203C3F4137203C3F4136203C3F41352096
:101500003C3F4134203C3F4133203C3F4132203C72
:101510003F4131203C3F41300A504F525442203C21
:101520003F4237203C3F4236203C3F4235203C3F43
:101530004234203C3F4233203C3F4232203C3F4239
:1015400031203C3F42300A504F525443203C3F43ED
:1015500037203C3F4336203C3F4335203C3F43341B
:10156000203C3F4333203C3F4332203C3F4331202B
:101570003C3F43300A504F525444203C3F443720B4
:101580003C3F4436203C3F4435203C3F4434203CE3
:101590003F4433203C3F4432203C3F4431203C3FD9
:1015A00044300A504F525445203C3F4537203C3F81
:1015B0004536203C3F4535203C3F4534203C3F45A7
:1015C00033203C3F4532203C3F4531203C3F4530B5
:1015D0000A3C2F5052453E3C68723E3C2F626F647D
:1015E000793E3C2F68746D6C3E0A0A6764656D6FC6
:1015F0002E68746D6C0005746578742F68746D6C5A
:101600000A0A3C68746D6C3E3C686561643E3C6DE2
:1016100065746120687474702D65717569763D22FA
:10162000436F6E74656E742D547970652220636FFC
:101630006E74656E743D22746578742F68746D6C79
:101640003B636861727365743D69736F2D3838351B
:10165000392D31223E3C6D65746120687474702DA3
:1016600065717569763D22526566726573682220E0
:10167000636F6E74656E743D2234223E3C2F686544
:1016800061643E0A3C626F647920746578743D231E
:10169000303030303030206267636F6C6F723D23C2
:1016A000453045304530206C696E6B3D233030301D
:1016B00030464620766C696E6B3D233830303038CA
:1016C0003020616C696E6B3D234646303030303ED1
:1016D0000A3C68723E3C703E5468697320776562CC
:1016E000736974652069732062726F75676874200E
:1016F000746F20796F75206279206120776562733D
:1017000065727665722074686174206973207275E1
:101710006E6E696E67206F6E2061205049433138CC
:101720004634353220636F6E6E6563746564207471
:101730006F20612033434F4D2033433530394220F1
:1017400065746865726E657420636172642E3C2FE7
:10175000703E0A3C703E42656C6F7720796F752051
:1017600063616E2073656520776869636820696EC0
:10177000707574206F662074686973205049433116
:1017800038663435322069732068696768203C699F
:101790006D67207372633D22312E676966223E2099
:1017A0006F72206C6F77203C696D67207372633DA8
:1017B00022302E676966223E2E3C2F703E3C6872B6
:1017C0003E0A3C5052453E0A504F525441203C691B
:1017D0006D67207372633D3C3F41372E6769663EFB
:1017E000203C696D67207372633D3C3F41362E6734
:1017F00069663E203C696D67207372633D3C3F41E2
:10180000352E6769663E203C696D67207372633DC3
:101810003C3F41342E6769663E203C696D6720730A
:1018200072633D3C3F41332E6769663E203C696DE3
:1018300067207372633D3C3F41322E6769663E20EC
:101840003C696D67207372633D3C3F41312E67698F
:10185000663E203C696D67207372633D3C3F4130BA
:101860002E6769663E0A504F525442203C696D67AC
:10187000207372633D3C3F42372E6769663E203CD1
:10188000696D67207372633D3C3F42362E6769661F
:101890003E203C696D67207372633D3C3F42352EAC
:1018A0006769663E203C696D67207372633D3C3F0B
:1018B00042342E6769663E203C696D67207372630F
:1018C0003D3C3F42332E6769663E203C696D672090
:1018D0007372633D3C3F42322E6769663E203C692D
:1018E0006D67207372633D3C3F42312E6769663EEF
:1018F000203C696D67207372633D3C3F42302E6728
:1019000069663E0A504F525443203C696D6720730C
:1019100072633D3C3F43372E6769663E203C696DEC
:1019200067207372633D3C3F43362E6769663E20F5
:101930003C696D67207372633D3C3F43352E676998
:10194000663E203C696D67207372633D3C3F4334C3
:101950002E6769663E203C696D67207372633D3C6B
:101960003F43332E6769663E203C696D6720737282
:10197000633D3C3F43322E6769663E203C696D679C
:10198000207372633D3C3F43312E6769663E203CC5
:10199000696D67207372633D3C3F43302E67696613
:1019A0003E0A504F525444203C696D672073726365
:1019B0003D3C3F44372E6769663E203C696D672099
:1019C0007372633D3C3F44362E6769663E203C6936
:1019D0006D67207372633D3C3F44352E6769663EF8
:1019E000203C696D67207372633D3C3F44342E6731
:1019F00069663E203C696D67207372633D3C3F44DD
:101A0000332E6769663E203C696D67207372633DC3
:101A10003C3F44322E6769663E203C696D67207307
:101A200072633D3C3F44312E6769663E203C696DE0
:101A300067207372633D3C3F44302E6769663E0AFF
:101A4000504F525445203C696D67207372633D3C92
:101A50003F45372E6769663E203C696D672073728B
:101A6000633D3C3F45362E6769663E203C696D67A5
:101A7000207372633D3C3F45352E6769663E203CCE
:101A8000696D67207372633D3C3F45342E6769661C
:101A90003E203C696D67207372633D3C3F45332EA9
:101AA0006769663E203C696D67207372633D3C3F09
:101AB00045322E6769663E203C696D67207372630C
:101AC0003D3C3F45312E6769663E203C696D67208D
:101AD0007372633D3C3F45302E6769663E0A3C2F7A
:101AE0005052453E3C68723E3C2F626F64793E3CEA
:101AF0002F68746D6C3E0A09696E666F2E68746D8E
:101B00006CC902746578742F68746D6C0A0A3C2184
:101B1000444F43545950452048544D4C2050554251
:101B20004C494320222D2F2F5733432F2F44544409
:101B30002048544D4C20342E3031205472616E7345
:101B40006974696F6E616C2F2F454E223E0A3C68A6
:101B5000746D6C3E0A3C686561643E0A3C6D657458
:101B60006120687474702D65717569763D22436FCC
:101B70006E74656E742D547970652220636F6E7477
:101B8000656E743D22746578742F68746D6C3B6368
:101B90006861727365743D69736F2D383835392DFE
:101BA00031223E0A3C7469746C653E5049433138B9
:101BB00066343532202B2033434F4D2033433530AC
:101BC0003942202D20576562736572766572202D2B
:101BD0003C2F7469746C653E0A3C6D657461206EBF
:101BE000616D653D224B6579776F72647322206366
:101BF0006F6E74656E743D225049433138663435DA
:101C0000322C203343353039422C2077656273659E
:101C100072766572223E0A20203C7374796C6520CE
:101C2000747970653D22746578742F637373223EF6
:101C30000A09613A686F7665727B636F6C6F723AFE
:101C40007265643B20746578742D6465636F72619E
:101C500074696F6E3A6E6F6E653B207D0A20203C82
:101C60002F7374796C653E0A3C2F686561643E0A87
:101C70000A3C626F647920746578743D22233030A9
:101C80003030303022206267636F6C6F723D2223E8
:101C900045304530453022206C696E6B3D22233043
:101CA00030303046462220766C696E6B3D222338F8
:101CB00030303038302220616C696E6B3D22234613
:101CC0004630303030223E0A3C68723E0A3C756C29
:101CD0003E0A3C6C693E0A596F752063616E20664E
:101CE000696E64206D6F726520696E666F0A3C6173
:101CF00020687265663D22687474703A2F2F77777A
:101D0000772E6A616E772E656173796E65742E62C7
:101D1000652F7069633138663435322D652E6874ED
:101D20006D6C22207461726765743D225F746F7000
:101D3000223E686572653C2F613E2E0A3C2F6C691D
:101D40003E0A3C6C693E0A4D65657220696E666F9D
:101D5000726D617469652076696E64206A650A3CFB
:101D60006120687265663D22687474703A2F2F771F
:101D700077772E6A616E772E656173796E65742E42
:101D800062652F7069633138663435322E68746D40
:101D90006C22207461726765743D225F746F7022DB
:101DA0003E686965723C2F613E2E0A3C2F6C693E8D
:101DB0000A3C2F756C3E0A3C68723E0A3C2F626FEB
:0E1DC00064793E0A3C2F68746D6C3E0A000088
:020000040030CA
:04000000FFF9FCFE0A
:02000600FAFFFF
:00000001FF
